:1000000012C02BC02AC029C028C027C026C025C0C6
:1000100024C023C022C021C020C01FC01EC01DC0DC
:100020001CC01BC01AC011241FBECFE5D4E0DEBF28
:10003000CDBF10E0A0E6B0E0E6E3F1E002C005903D
:100040000D92A036B107D9F710E0A0E6B0E001C0EC
:100050001D92A036B107E1F760C0D2CF40E050E07A
:100060004817590768F420E030E0275E3F4F60E70B
:100070002E343607D0F34F5F5F4F4817590798F378
:10008000089580B7846080BF87B38F6387BB88B3D0
:10009000817E816288BB84B3837C836084BB85B3AB
:1000A000807C85BB81B384EF81BB82B380E282BB5D
:1000B000089581B3806381BB82B3806382BB87B3C1
:1000C000806387BB88B38F7C88BB87B3866087BB20
:1000D00088B3897F88BB8FB581EA8FBD8EB5827268
:1000E00082608EBD1BBC1ABC19BC18BC82B38F7E4B
:1000F00090E2892B82BB88B38F7E892B88BB0895C1
:1001000087B18377836687B986B1867D866C86B929
:100110003699FECF85B199270895CFE5D4E0DEBFAB
:10012000CDBF85B5887F85BDACDFC3DFE9DF99270B
:060130009BBD8ABDFBCF60
:00000001FF
